:020000040000FA
:0400000081EF01F09B
:08000800E8CF05F0D8CF06F0A7
:10001000E0CF07F00001E9CF0DF0EACF08F0E1CF23
:1000200009F0E2CF0AF0D9CF0BF0DACF0CF0F3CF22
:1000300014F0F4CF15F0FACF16F000C00FF001C0A5
:1000400010F002C011F003C012F004C013F09DAA1A
:100050002DEF00F09EBA9CEF00F00FC000F010C032
:1000600001F011C002F012C003F013C004F00DC083
:10007000E9FF08C0EAFF09C0E1FF0AC0E2FF0BC0C8
:10008000D9FF0CC0DAFF14C0F3FF15C0F4FF16C08F
:10009000FAFF05C0E8FF07C0E0FF06C0D8FF100068
:1000A000F2CF0EF0F29EF76ABA0FF66E000EF7224C
:1000B0000900F5500EBEF28E1200496E6974696136
:1000C0006C697A696E6720506F727420420A0D0065
:1000D000F2CF0EF0F29EF76AEA0FF66E000EF722EC
:1000E0000900F5500EBEF28E1200436F6E6669670E
:1000F0007572696E672052462D3234470A0D000032
:10010000F2CF0EF0F29EF76A1A0FF66E010EF7228A
:100110000900F5500EBEF28E12004F4B210A0D0061
:100120009EAAFED7ABCF18F0AECF01F018A202D036
:10013000AB98AB880000000CF3DF01C029F0295018
:10014000120A01E025D0ECDF0150340802E0000E75
:1001500001D0010E2B6EE4DF0150560802E0000EC4
:1001600001D0010E2B142D6EDBDF0150780802E068
:10017000000E01D0010E2D142F6ED2DF0150900819
:1001800002E0000E01D0010E2F14D8A4FF0000D011
:100190009E9A2DEF00F0EA6A230EE96EEF500FE011
:1001A000030E016E006A002EFED7012EFBD73C0E17
:1001B000006E002EFED700000000EF2EF1D7000CDD
:1001C000070E276E266A265007081DE3939A8A9A1F
:1001D00027502706286E25C000F02850016E04E045
:1001E000D8900032012EFCD700A003D093988A88C3
:1001F00002D093988A9800000000939A8A8A00009F
:100200000000262AE0D7000C93968A96939E8A9E39
:10021000939A8A9A93988A98030E236EBCDF939ED2
:100220008A8E080E006E002EFED7300E256EC8DFB7
:10023000300E256EC5DF256AC3DF256AC1DF256A5A
:10024000BFDF420E256EBCDF420E256EB9DF256A88
:10025000B7DF256AB5DF256AB3DF420E256EB0DF52
:10026000420E256EADDF430E256EAADF6F0E256EA2
:10027000A7DF810E256EA4DF938893968A96939EBE
:100280008A9E939A8A9AF3EF01F093968A96939EA8
:100290008A8E080E006E002EFED793988A98939A45
:1002A0008A8A00000000939A8A9A00000000939EB8
:1002B0008A9E939A8A9A05EF02F093968A86080E90
:1002C000006E002EFED7420E256E7ADF420E256E9E
:1002D00077DF236A235005080EE3036A2350190FC2
:1002E000E96E000E0320EA6EEFCF24F024C025F063
:1002F00067DF232AEFD793968A96939A8A9A4BEFD1
:1003000002F0F86AD09E0D8EEA6AE96AB8862A0E73
:10031000AF6E000EB06E260EAC6E900EAB6EC1507E
:10032000C00B0F09C16E070EB46E186A7F0E1F6EE8
:10033000206EC150C00B0C09C16EC090C082C08439
:10034000C08EC280880ED56ECD6A000ECA6E7F0E3A
:10035000CB6EB150480BB16EB70EB1169484BD6A26
:10036000BD6AB1169482BA6ABA6A9D8AC00EF21248
:10037000236A235095DE232A006E00509EA8FED7E4
:10038000AD6E130E235CF5E1030E246E2E0E9EA8B7
:10039000FED7AD6E242EFAD70A0E9EA8FED7AD6EFC
:1003A0000D0E9EA8FED7AD6EF18EF296236A2350F5
:1003B0008FDE232A006E00509EA8FED7AD6E120E6F
:1003C000235CF5E1030E246E2E0E9EA8FED7AD6EC3
:1003D000242EFAD70A0E9EA8FED7AD6E0D0E9EA84B
:1003E000FED7AD6E11D77F0E196E1A6E1B6E1C6E86
:1003F000236A235085DE232A006E00509EA8FED774
:10040000AD6E050E235CF5E140D7010E236EC3DE11
:10041000000E016EC250C30B0110C26E100E006EB2
:10042000002EFED70000C282C2B2FED7C3CF21F099
:10043000C4CF22F022C019F021C01AF0040E016EC0
:10044000C250C30B0110C26E100E006E002EFED7FC
:100450000000C282C2B2FED7C3CF21F0C4CF22F0C7
:1004600022C01BF021C01CF0080E016EC250C30B4D
:100470000110C26E100E006E002EFED70000C28268
:10048000C2B2FED7C3CF21F0C4CF22F022C01DF0EC
:1004900021C01EF012D794948B74320E236E7BDE33
:0404A000B7D70300C7
:00000001FF
